:020000020000FC
:1000000038CF189518951895C8CD39C918951895F1
:1000100098CC18951895189518951895DBC51895CE
:100020001895000000000000000E111B1115110EA4
:100030000E1F151F1F1B0E0A1B1F1F0E0E04040E82
:100040001F1F0E04000E04151F150404040E0E1FBE
:100050001F040E0000040E0400001F1F1B111B1FB5
:100060001F00040A110A04001F1B1111111B1F039A
:1000700003040E11110E0E11110E040E04060505D7
:10008000040418180C0A0909091B1B00040E1B0E96
:100090000400080C0E0F0E0C0802060E1E0E0602BF
:1000A000040E0404040E040A0A0A0A0A000A1F1DA8
:1000B0001D050505050F100E110E011E0000001F85
:1000C0001F0000040E040E04000E040E04040404B9
:1000D0000404040404040E040000021F02000000D3
:1000E00000081F0800000000101010101F00000A78
:1000F0001F0A00000000040E1F00000000001F0E79
:1001000004000000000000000004040404040004D3
:100110000A0A0A000000000A0A1F0A1F0A0A040F3E
:10012000140E051E041819020408130308141409F8
:1001300015120D060204000000000204080808045D
:10014000020804020202040804150E040E1504003D
:1001500004041F0404000000000006020400000064
:100160001F00000000000000000606000102040855
:1001700010000E11111111110E040C040404040ED0
:100180000E11010204081F1F02040201110E0206D3
:100190000A121F02021F101E0101110E0E11101E65
:1001A00011110E1F0102020404040E11110E11118F
:1001B0000E0E11110F01110E000C0C000C0C0000A2
:1001C0000C0C000C04080204081008040200001FB4
:1001D000001F0000080402010204080E11010204BD
:1001E00000040E11171517100E040A11111F11111A
:1001F0001E11111E11111E0E11101010110E1C12C5
:10020000111111121C1F10101E10101F1F10101E94
:100210001010100E11101711110F1111111F1111C3
:10022000110E04040404040E0F02020202120C1147
:100230001214181412111010101010101F111B1589
:1002400015151111111119151311110E111111118B
:10025000110E1E11111E1010100E11111115120D7C
:100260001E11111E1412110E11100E01110E1F0479
:1002700004040404041111111111110E11111111B2
:10028000110A041111111515150A11110A040A1188
:100290001111110A040404041F01020408101F0EA6
:1002A00008080808080E001008040201000E0202E7
:1002B0000202020E040A110000000000000000000B
:1002C000001F0C08040000000000000E010F110FB9
:1002D00010101E1111111E00000F1010100F01013F
:1002E0000F1111110F00000E111F100E0304041F37
:1002F00004040400000F110F010E10101619111143
:100300001104000C0404040E0200060202120C0088
:100310001012141814120C04040404040E00000A31
:10032000151511110000161911111100000E1111EF
:10033000110E00001E111E10100000070907010118
:1003400000000B0C08080800000E100E011E04042B
:100350001F040404030000111111130D00001111FA
:10036000110A040000111115150A0000110A040AEF
:1003700011000011110F010E00001F0204081F06DA
:10038000080810080806040404000404040C02020F
:100390000102020C1926000000000000000000000D
:1003A000000000000000000000000000000000004D
:1003B0001818000708080711040015000411150A91
:1003C000150A150A150000000000000000000000DA
:1003D0000000000000000000000006091C081C09C5
:1003E0000600000000000000000000000000000007
:1003F00000000000000000000000000000000000FD
:1004000000000000000000000000000000000000EC
:1004100000000000000000000000000000000000DC
:1004200000000000000000000000000000000000CC
:1004300000000000000000000000000000000000BC
:1004400000000000000000000000000000000000AC
:10045000001F0404111B1511000000000000000023
:10046000000000000000000000000000000000008C
:10047000000000000000000000000000000000007C
:10048000000000000000000000000000000000006C
:10049000000000000000000000000000000000005C
:1004A000000000000000000000000000000000004C
:1004B000000000000000000000000A1F101C1C10BB
:1004C0001F0E11151915110E0E11101C10110E0012
:1004D000000000000000000000000000000000001C
:1004E000000000000E111D1B1D1B0E0A001F04043E
:1004F000041F0000000000000004041F0404001F8B
:100500000E04040404040E04000C0404040E000091
:1005100000000000000000000000000000000000DB
:10052000000006000000000000000A000E111F106D
:100530000E1313121A16121200000E111C110E00C7
:1005400000000000000000000000000000000000AB
:1005500000000000000000000000000A000C04047D
:10056000040E0709111F1111111E10101E11111E6A
:100570001E11111E11111E1F111010101010060A4D
:100580000A0A0A1F111F10101E10101F1515150E34
:100590001515150E11010601110E11111113151962
:1005A0001115111113151911111214181412110724
:1005B000090909090911111B151111111111111145
:1005C0001F1111110E11111111110E1F1111111105
:1005D00011111E1111111E10100E11101010110EFC
:1005E0001F1504040404041111110F01110E0E153E
:1005F00015150E040411110A040A11111212121217
:10060000121F01111111110F0101151515151515E5
:100610001F15151515151F0118080E0909090E11CA
:1006200011191515151910101E1111111E0E110199
:100630000701110E1215151D1515120F11110F05B9
:10064000091100000E010F110F0F08040E11110EF9
:100650000C12141E11110E00001E12101010000EAC
:10066000010F11110E00000E111F100E00001515C4
:100670000E151500000E1106110E000011131519AC
:100680001100041113151911000011121C12110090
:100690000007090909190000111B151111000011AB
:1006A000111F111100000E1111110E00001F111168
:1006B000111100001E11111E1000000E1110110E5C
:1006C00000001F04040404000011110F011E0000AB
:1006D0000E15150E040000110A040A110000121272
:1006E000121F01000011110F010100001515151551
:1006F0001F00001515151F01000018080E090E0037
:10070000001119151519000010101E111E00000E01
:100710001107110E000012151D151200000F110F08
:1007200005192020202020202020202020202020EB
:1007300020202020202020202020202020202020B9
:100740002020202122232425262728292A2B2C2D4E
:100750002E2F4F3132333435363738393A3B3C3D22
:100760003E3F404142434445464748494A4B4C4D31
:100770004E4F505152535455565758595A5B2F5D4E
:100780005E5F606162636465666768696A6B6C6D11
:100790006E6F707172737475767778797A28D12953
:1007A000E97F060704FFFF85868702898A8B8C8D87
:1007B0008E8F902727CBCA95969798019A9B9C9DE0
:1007C0009E9FA0A1A2A3A4A5A6A7A2A9AAABACADD7
:1007D000AEAFB003B2B3B4B5B6B7B54EBABBBCBDDD
:1007E000BEBF41A042A1E045A3A4A5A64BA74D488A
:1007F0004FA8504354A9AA58E1ABACE2ADAE05AF47
:10080000B0B161B2B3B4E365B6B7B8B9BABBBCBDF9
:100810006FBE7063BF79E478E5C0C1E6C2C3C4C5EA
:10082000C6C7868F98A1AA0000000000858E97A0F9
:10083000A90000000000838C959EA70B3331320085
:10084000848D969FA81B3937380F879099A2AB11DA
:100850000403011088919AA3AC141A090615808923
:10086000929BA413050C0712818A939CA50D363424
:100870003508828B949DA60002301900B3BCC5CE0A
:10088000D70000000000B2BBC4CDD60000000000BD
:10089000B0B9C2CBD40B33313200B1BAC3CCD51B03
:1008A0003937380FB4BDC6CFD81104030110B5BE17
:1008B000C7D0D9141A090615ADB6BFC8D113050C97
:1008C0000712AEB7C0C9D20D36343508AFB8C1CAA9
:1008D000D3000230190098A1C5CED7000000000057
:1008E00097A0C4CDD60000000000959EC2CBD40BCB
:1008F00033313200969FC3CCD51B3937380F99A2BC
:10090000C6CFD811040301109AA3C7D0D9141A096D
:100910000615929BBFC8D113050C0712939CC0C942
:10092000D20D36343508949DC1CAD3000230190067
:100930006770793A7B0000000000666F782D3D00FB
:1009400000000000646D765F400B33313200656E4D
:1009500077222A1B3937380F68717A3C7D110403DE
:10096000011069725B3E20141A090615616A73B1A1
:100970003F13050C0712626B745D2F0D363435087A
:10098000636C755EB900023019004750593B28006E
:1009900000000000464F582B260000000000444D88
:1009A000565F240B33313200454E5722251B393711
:1009B000380F48515A2C29110403011049525B2E5B
:1009C00020141A090615414A53822113050C0712F7
:1009D000424B545D220D36343508434C555E23009E
:1009E00002301900E6EFF83A7B0000000000E5EE67
:1009F000F72D3D0000000000E3ECF5FE400B333125
:100A00003200E4EDF6FF2A1B3937380FE7F0F93CE6
:100A10007D1104030110E8F1FA3E20141A090615AD
:100A2000E0E9F2FB3F13050C0712E1EAF3FC2F0D9E
:100A300036343508E2EBF4FDB90002301900C6CFB8
:100A4000D83B280000000000C5CED72B26000000B0
:100A50000000C3CCD5DE240B33313200C4CDD6DF49
:100A6000251B3937380FC7D0D92C291104030110A1
:100A7000C8D1DA2E20141A090615C0C9D2DB2113F9
:100A8000050C0712C1CAD3DC220D36343508C2CB9F
:100A9000D4DD2300023019008813A00FAC0DB80B71
:100AA000C409D007DC05E803F401FA0020534854D8
:100AB0005249482D5052494E5420444953504C41BC
:100AC0005920534D3830372E333120762E312E3287
:100AD000205255532044314E534D3830372E333148
:100AE00020762E312E32205255532044324E0B0B9D
:100AF0000B0B0B0B0B0B0A0A0A0A0A0A0A0A090952
:100B000009090909804020100804020180402010D2
:100B100008040201804020100804000000000000CA
:100B200000000101010101010101020202020202B1
:100B300001020408102040800102040810204080B7
:100B40000102040810206D01CC0000000091CC00CF
:100B500008950FEF0ABB04E10BBB00E407BB0FE0F5
:100B600008BB01E004BB0FEF05BB01BB02BB07E004
:100B700006B907B99F9905C001E00093CC00DAD708
:100B800009C008E101BD05E001BD02E00093CC0011
:100B9000A3D236D303D080D67894089500E002BF64
:100BA0000DE701BF0BE003BF09B7016009BF0EEFFE
:100BB00002BBA89A00E00093D700089530E02223FA
:100BC00039F000FD05C01695079533953217C8F327
:100BD000032F0895BA93AA938A93FA93EA933A92C9
:100BE0002A921A920A927A936A935A934A933A9360
:100BF0002A931A930A938FB7ADECB0E00D911C9134
:100C00001197012B51F00D91015010401C930E9340
:100C100011961197012B09F46AD6FD010281138107
:100C2000012B49F002810150104002831383012BF4
:100C300011F400E0008B04811581012B59F408EEBA
:100C400013E00483158301E0128510271287012F1A
:100C500093D205C004810150104004831583FD0127
:100C600006811781012B29F006810150104006836F
:100C7000178303850023F1F000890023D9F400E0F5
:100C800003870189033031F400ED17E002831383F9
:100C90000CE10FC0043031F400ED17E00283138340
:100CA0000DE107C0023031F400ED17E00283138339
:100CB0000EE1008B0485005049F00A9561F10A9518
:100CC00009F45EC00A9509F494C033C026B32F70AE
:100CD00003B310E00E77000F000F111F000F111F5C
:100CE000022B0F3F134089F4979904C00FEF02BB0A
:100CF000A898A4C0A89904C00EEF02BBA89A9EC0F1
:100D000002B3000F016002BB99C0048503950487FC
:100D10000AE0058793C026B32F7003B310E00E7767
:100D2000000F000F111F000F111F022B0F3F134068
:100D300019F400E0048782C005850A950587002321
:100D400009F07CC02AE046B34F7003B310E00E7781
:100D5000000F000F111F000F111F042B009510959D
:100D60002DDFFD01068729E002B310E0A89911E00C
:100D70000095109523DFFD01078704850395DACFE1
:100D800000ED17E002831383278530E00AE0029F1D
:100D900026854091540146FD0DC043FF08C047FF22
:100DA00003C0E6EDF8E017C0ECE7F8E014C0E2E2BB
:100DB000F8E011C045FD08C043FF03C0EEE3FAE0D0
:100DC0000AC0E4EEF9E007C043FF03C0EAE8F9E037
:100DD00002C0E0E3F9E0E00DF11DE20FF31F049122
:100DE000FD01008B0089018B308731870AEF058771
:100DF000C4CF26B32F7003B310E00E77000F000F9F
:100E0000111F000F111F022B0F3F134079F40585AE
:100E10000A950587002391F400E004870085118579
:100E20000D3D154058F001E0038708C00AEF058723
:100E3000008511850F5F1F4F008711878FBF0991B4
:100E40001991299139914991599169917991099013
:100E5000199029903990E991F9918991A991B991C5
:100E6000189504EF11E0EDECF0E000831183089594
:100E700000E0EDECF0E0008301830895EDECF0E09C
:100E800000E002830383008B08952FB7F894EDEC04
:100E9000F0E006811781012B11F001E001C000E0B4
:100EA0002FBF08952FB7F894EDECF0E00683178379
:100EB0002FBF089539983A98389A0BBB000000006C
:100EC00038980AEC0A95F1F700C0089539983A98D5
:100ED000389A0BBB0000000038980895399AEBCF80
:100EE000399AF5CFE7DF0FE11EE401501040E9F732
:100EF00000C0000006E0DEDF0FE11EE401501040FC
:100F0000E9F700C000000CE0D5DF0FE11EE401505E
:100F10001040E9F700C0000008E4CCDF0FE1DEDF9D
:100F200009E4C8DF04E0DADF0AE4C4DF04E0D6DF66
:100F30000BE4C0DF01E1D2DF0CE4BCDF0BE1CEDF6C
:100F40000DE4B8DF05E1CADF0EE4B4DF01E1C6DF7E
:100F50000FE4B0DF00E0C2DF00E5ACDF06E0BEDF9B
:100F600001E5A8DF09E0BADF02E5A4DF0CE1B6DFA6
:100F700003E5A0DF08E0B2DF04E59CDF0CE1AEDFB3
:100F800005E598DF09E0AADF06E594DF06E0A6DFC5
:100F900007E590DF00E0A2DF08E58CDF04E09EDFDC
:100FA00009E588DF04E09ADF0AE584DF0FE196DFD8
:100FB0000BE580DF04E092DF0CE57CDF04E08EDFF0
:100FC0000DE578DF00E08ADF0EE574DF0FE186DFF4
:100FD0000FE570DF00E082DF00E66CDF08E17EDF16
:100FE00001E668DF08E17ADF02E664DF06E076DF2B
:100FF00003E660DF09E072DF04E65CDF08E06EDF35
:1010000005E658DF09E06ADF06E654DF06E066DF42
:1010100007E650DF00E062DF08E64CDF00E15EDF5C
:1010200009E648DF00E15ADF0AE644DF0EE156DF59
:101030000BE640DF01E152DF0CE63CDF01E14EDF71
:101040000DE638DF01E14ADF0EE634DF0EE146DF70
:101050000FE630DF00E042DF00E72CDF00E03EDF9C
:1010600001E728DF00E03ADF02E724DF00E036DFB7
:1010700003E720DF00E032DF04E71CDF00E02EDFC3
:1010800005E718DF00E02ADF06E714DF00E026DFCF
:1010900007E710DF00E022DF08E70CDF00E01EDFDB
:1010A00009E708DF00E01ADF0AE704DF00E016DFE7
:1010B0000BE700DF00E012DF0CE7FCDE00E00EDFF4
:1010C0000DE7F8DE00E00ADF0EE7F4DE00E006DF01
:1010D0000FE7F0DE00E002CF0FEF19EF0000015044
:1010E0001040E1F700C000C008E3E4DE0FE11EE4B9
:1010F00001501040E9F700C0000008E3DBDE07E51F
:1011000012E001501040E9F700C0000008E3D2DE11
:101110000FE113E001501040E9F700C0000008E3C0
:10112000C9DE0FE11EE401501040E9F700C00000E5
:1011300008E0C0DE0FE11EE401501040E9F700C0F6
:10114000000001E0CFCEAD01EBE0F1E024892160A9
:10115000248BDF0127E0F80131918F013D932A951F
:10116000D1F7DA010895AD01EBE0F1E024892260C6
:10117000248BA2E1B1E0EECF00931E010895BA9353
:10118000AA939A93382E2FB6F894B801842FABE027
:10119000B1E0FD010589002311F000E02BC00FED47
:1011A00010E09CE242E257E0FB010190BF011124F4
:1011B000400D511DFA014491F80141938F019A9518
:1011C00089F78D01025F1F4F43E0F90151919F01A3
:1011D000F80151938F014A95C1F7882311F08D32A0
:1011E00018F0FD01118A05C001E0FD01018B8A950F
:1011F000828B01E02FBE832D9991A991B991089519
:1012000000E010E00DBD0CBD08EC19BD08BD1FBD10
:1012100003E00EBD09B7006209BF0895EBE0F1E0FD
:10122000008D002329F000E0008F09B7006209BF9C
:1012300008952497402FEBE0F1E0068508830785A9
:10124000098300890A83088119812A813B8155E03D
:10125000459F402D1BD6202F2F7100E024FB0EF45C
:1012600001E023FB0EF4026022FB0EF4046021FB7C
:101270000EF4086020FB0EF4006124960895BA93E2
:10128000AA938A93FA93EA933A922A921A920A922A
:101290007A936A935A934A933A932A931A930A93A6
:1012A0008FB700E010E00DBD0CBDABE0B1E0FD017B
:1012B0000189002351F00389002339F00FE52289C9
:1012C00030E0F901E152FF4F0083FD0107892FED66
:1012D00030E0200F311F16891050A9F01A9571F1D6
:1012E0001A9509F441C01A9509F44DC01A9509F4EC
:1012F00093C01A9509F4A4C01A9509F4ECC01A9584
:1013000009F426C133C111E0158B002319F400E85C
:10131000DDDD05C021503040F9010081E1DDFD0136
:1013200007890395078B073108F423C100E0078B79
:1013300006890395068B00E0058B1BC111E0158B18
:10134000002319F400ECC2DD03C0F9010589C8DDF2
:10135000FD0107890395078B073108F40AC10AE3E9
:10136000BFDD00E0FD01E3CF002319F406E9AEDDA7
:1013700002C000E0B5DDFD0107890395078B02304F
:1013800008F4F7C0D3CF002319F400E49FDD3EC07A
:10139000013031F401E0058B00E04BDFA1DD36C008
:1013A000023011F401E4F2CF033011F401E0F5CF83
:1013B000043011F402E4EACF053011F402E0EDCF7D
:1013C000063011F403E4E2CF073011F403E0E5CF77
:1013D000083011F404E4DACF093011F404E0DDCF71
:1013E0000A3021F400E0058B05E4D0CF0B3011F476
:1013F00000E0D4CF0C3011F406E4C8CF0D30C1F3B7
:101400000E3011F407E4C2CF0F3091F3FD010789CC
:101410000395078B0031B4CF048900FF07C00E7F0E
:10142000048B06890395068B00E0A2C001FF05C06E
:101430000D7F048B06890E5FF6CF07E0068B99C0FF
:10144000002319F400E742DD3CC0013011F40C9197
:1014500037C0023011F401E7F6CF033011F40181F7
:101460002FC0043011F402E7EECF053011F40281F1
:1014700027C0063011F403E7E6CF073011F40381EB
:101480001FC0083011F404E7DECF093011F40481E5
:1014900017C00A3011F405E7D6CF0B3011F40581DF
:1014A0000FC00C3011F406E7CECF0D3011F40681D9
:1014B00007C00E3011F407E7C6CF0F3011F400E07B
:1014C0000FDDFD0107890395078B003108F451C03A
:1014D00000E0078BB2CF002311F408E7B4CF01304E
:1014E00011F40781EDCF023011F409E7ACCF0330DE
:1014F00011F40085E5CF043011F40AE7A4CF0530DC
:1015000011F40185DDCF063011F40BE79CCF0730D5
:1015100011F40285D5CF083011F40CE794CF0930CF
:1015200011F40385CDCF0A3011F40DE78CCF0B30C9
:1015300011F40485C5CF0C3011F40EE784CF0D30C3
:1015400011F40585BDCF0E3009F0B7CF0FE77BCF83
:10155000018D0395018F053138F000E0018F01E026
:10156000008F09B70F7D09BF00E068CF00E0068B50
:10157000078B8FBF099119912991399149915991FF
:10158000699179910990199029903990E991F9918F
:101590008991A991B9911895A89522E531E005E2C4
:1015A00011E07FD10FE91FE001501040E9F700C0C2
:1015B000000005E211E019D1C9DA02304091510171
:1015C00022E531E005E211E019F4D9DD27DE01C0A2
:1015D000C0D296D1002301F3FFCF01E00093550163
:1015E000089501E00093570100E010E05BCC009308
:1015F0005801089500935C01089500935B010895DC
:10160000BD01D901FA012481222391F426E1F801D8
:1016100031918F013D932A95D1F720E005C030E24A
:10162000FD013193DF012395FA0136812317B8F3C9
:101630002481213079F420E003C030E23D932395EA
:1016400036812317D0F326E1F80131918F013D93C4
:101650002A95D1F7FA0106810A5EDB010895AC01F3
:10166000F8013081E22FF0E03197E13020E0F2071D
:1016700044F0CF01F801218120830F5F1F4F0197B4
:10168000C9F7F8013083CA010895BD01AC01822F6A
:1016900090E0020F191F01501040F80120810197BE
:1016A000813030E093074CF0DC01F8013291F80111
:1016B0003083015010401197C1F7F8012083CA010F
:1016C000DB0108959A938A93C80100915A01013071
:1016D00011F0002341F445E551E02DE531E08C01A6
:1016E0008FDF0093B50100915A01023011F0002301
:1016F00049F445E551E029E831E046968C0180DF68
:101700000093B601899199910895E5E5F1E013817F
:10171000012F0F7039F000E00483012F017149F0AF
:1017200000E00FC0012F007F11F001E0F5CF00E0D5
:101730000895012F027211F001E003C01474B9F38F
:1017400002E005830681073190F707810A3078F7B8
:1017500001E00895BA93AA939A938A93D80195DBEE
:101760000023F1F5CD0100915A01013011F0002361
:1017700091F42091B5010091590100230DE511E08C
:1017800011F46DDF01C081DFEDE5F1E006E11191BB
:101790001D930A95E1F700915A01023011F00023E0
:1017A000A1F42091B60100915901002309E811E04C
:1017B00011F455DF01C069DFDC015696E9E8F1E07C
:1017C00006E111911D930A95E1F7E8E9FAE000912D
:1017D0005C0112E0019FE00DF11D0591149162DBA7
:1017E00089919991A991B9910895BA93AA939A93DD
:1017F0008A93C801A5E5B1E0FD010281002329F02B
:1018000000E002830C9301831FC00C910023B9F008
:1018100000E00C937ADF0023B9F08C0153DF08E974
:101820001AE0FD01278132E0239F000D111DF80110
:101830000591149137DB01E0FD01018303C00181B3
:10184000002311F08C0186DFCBCFBA93AA939A9331
:101850008A938CEA9AE0A5E2B1E006E1FC011591D9
:10186000CF011D930A95D1F782EC9AE06FD902302F
:1018700011F488ED9AE0ABE3B1E006E1FC011591CB
:10188000CF011D930A95D1F789919991A991B991A9
:1018900008955FD9DADF80CE0FEF0FB900EC0DB9F4
:1018A00008951B2E2A2E0FB6F894A801E7EBF1E05D
:1018B00003810023C1F00FEE11E06CE2D8017D91AD
:1018C0008D01DA017D93AD016A95C1F70BE112E05C
:1018D00043E0D8015D918D01D9015D939D014A9549
:1018E000C1F700E003830FBEA22DB12D0895E7EBF1
:1018F000F1E000E000830283BBDA0FEF0FB9089537
:101900001FB7F894E7EBF1E000810023B9F40481FC
:10191000B69907C0002329F401E0048303E005839E
:101920000DC0002359F0B69B03C000E0048307C03C
:1019300005810A95058311F401E0F8CF00E01FBF8F
:1019400008954A92BA93AA939A938A93FA93EA9340
:101950003A922A921A920A927A936A935A934A93E3
:101960003A932A931A930A934FB60EB12FB1067089
:10197000B1F0BDDF4FBE099119912991399149917B
:101980005991699179910990199029903990E9912B
:10199000F99189919991A991B99149901895ADEBD7
:1019A000B1E087EB91E0FC01428150E08D01040F32
:1019B000151F3081332341F03A95E1F03A9509F44F
:1019C00052C03A95A9F1D5CF2B3121F401E0008323
:1019D0000FE20AC02D3121F403E0008308E004C0C7
:1019E0002C3139F602E0008301830091DD000FB94C
:1019F00038DAC0CF31813A953183F8012083FC0178
:101A00000281039502835FB90181002309F0F0CFC1
:101A10000FEE11E09D014FE2F90151919F01F80194
:101A200051938F014A95C1F701E0FC010383A1CFD7
:101A300031813A953183F8012083FC0102810395BD
:101A400002835FB90181002399F60C91002319F0FC
:101A50000A9529F08ECF11968D0175DB8ACF1196EC
:101A60008D0181DB86CF31813A953183F801208366
:101A7000FC010281039502835FB90181013029F4E1
:101A80000C91003121F662D80FB9FC0101810023CD
:101A900009F0AECFFD0101811C911A5059F01A9541
:101AA000C9F11A95F1F11A95F1F1125081F11A95D7
:101AB000E1F15FCF002349F4EFEEF1E00CE210E238
:101AC00011930A9509F455CFFACF013049F4EFEE9E
:101AD000F1E006E110E211930A9509F44ACFFACF3A
:101AE000023049F4E5E0F2E006E110E211930A95D4
:101AF00009F43FCFFACF033009F03BCFEBE1F2E03E
:101B000003E010E211930A9509F433CFFACF009362
:101B100051012FCF002311F464DD2BCF68DD5DDD93
:101B200028CF6BDD26CF66DD24CF002309F021CF3F
:101B3000A5D91FCF00E010E00DBD0CBD04EB1BBD0F
:101B40000ABD1FBD0BE00EBD09B7006409BFD89ADE
:101B500008955B2F6A2FD801EFEDF0E00CE21D91A4
:101B600011930A95E1F7A9E1B1E003E0F9011191C0
:101B70009F011D930A95D1F7442311F04D3220F0B7
:101B800000E000931C0106C001E000931C014A958F
:101B900040931D01A62FB52F0895BA93AA939A9347
:101BA0008A93FA93EA933A922A921A920A927A9331
:101BB0006A935A934A933A932A931A930A933FB695
:101BC000DC9AAEE1B2E020E00EEE1AE0FD01428DBB
:101BD00050E0040F121FF801049110E0FD01E00F26
:101BE000F21F2687DB9AFD01028D0395028F0631D5
:101BF00008F0228F228D30E0E4E0FBE0E20FF51FD9
:101C00004491EEEEFAE0E20FF51F0491FD01E00FC2
:101C1000F51F4687EAE1FBE0E20FF51F0491F801AA
:101C2000E75EFE4F0081E0E3FBE0E20FF51F149159
:101C3000102311F011E001C010E0DB980000DC98E7
:101C4000FD01028D802F90E04FED50E0400F531FBB
:101C5000FA016081603871F42BE031E0BD01E7E00A
:101C60000E2EF90111909F01FB011192BF010A9400
:101C700019F1F7CF613871F422E131E0BD01E7E0FD
:101C80000E2EF90111909F01FB011192BF010A94E0
:101C900099F0F7CF22E230E0262E67E0629D200D1A
:101CA000311DBD01E7E00E2EF90115909F01FB01EA
:101CB0001192BF010A94C1F7FA016689603879F47C
:101CC0002BE031E0AD01495F5F4F67E0F9017191B1
:101CD0009F01FA017193AF016A9521F1F7CF613845
:101CE00079F422E131E0AD01495F5F4F67E0F9012E
:101CF00071919F01FA017193AF016A9599F0F7CF45
:101D000022E230E047E0469F200D311DAD01495FE2
:101D10005F4F67E0F90175919F01FA017193AF017F
:101D20006A95C1F720911C012223F1F020911E0138
:101D30002223D1F020E030E040911D01401709F44A
:101D40009D0150E046964817590719F49D01295FF7
:101D50003F4F022F032B41F006E0F90151939F0101
:101D60000A95D9F70FE10083FD0121810C91000F45
:101D7000000F000F322F36953695302B368B0381AE
:101D800030E4239F3281330F3029202F22952F708A
:101D9000232B258B0295007F24812695202B248BD5
:101DA0000681248120FB20E027F93581330F330F92
:101DB000322B202F269526952695232B238B0295B3
:101DC000007F000F2781202B228B21850085000FAB
:101DD000000F000F322F36953695302B318B03854F
:101DE00030E4239F3285330F3029202F22952F7026
:101DF000232B208B0295007F24852695202B278777
:101E0000048500FB00E007F92585220F220F202B17
:101E10002687112319F0022F016006871E969D0167
:101E20000CE0F90141919F0118E0DA9840FB16F4AB
:101E3000D99A01C0D998DA9A46951A95B1F70A95B8
:101E4000002379F73FBE0991199129913991499160
:101E50005991699179910990199029903990E99156
:101E6000F99189919991A991B99118950000889556
:101E7000FECF0BEC0DBF00E00EBFC0E9D0E00ED0EE
:101E8000002309F01BD005DDF1DFF0CF4A952AF0E1
:101E90003695279517950795F9CF089501E0089590
:101EA00020E006D0E9F70895259102D0E9F70895DA
:101EB0002D9301501040202F212B089586E49BE0A4
:101EC000FC0105911491FC013296A591B491FC019D
:101ED000349625913491422F432B19F0F901E4DF18
:101EE00001C0DEDF06961BE08C34910748F30895AD
:0400000300000000F9
:00000001FF
